:020000040000FA
:02000000A8282E
:08000800072CA30121082218B6
:10001000A3070310A20C0310A10DA208031D0628BC
:1000200008002208A10708002608A4070318A50A4B
:100030002708A50708002208A1050800A20803193F
:100040000800A3010130AA000310AA0D0310A20D9D
:10005000A21F24282208A10203183028A107322851
:100060002A08A3070310A20C0310AA0C031C2A28B9
:100070000800A608031D3F28A7080319080001303F
:10008000AA00AB01A801A9010310AA0DAB0D031032
:10009000A60DA70DA71F442860200318512869202A
:1000A00057282A08A8070318A90A2B08A90703102C
:1000B000A70CA60C0310AB0CAA0C031C4C280800C0
:1000C0002708AC002608A402031CAC0A2C08A502D1
:1000D00008002608A4070318A50A2708A507080092
:1000E0002108A202031D003401342108A202031CCE
:1000F000003401343408B30408003408B3050800A0
:100100003808B6070318B70A3908B7070800B40952
:1001100008003408B30708003308B402031C003495
:1001200001343308B402031D003401343608B80228
:10013000031D00343708B902031D003401343608AA
:10014000B8023708031C370FB902031C003401340E
:10015000831203138501831603139B0107309C0050
:1001600000308500831203138601831603130030C9
:10017000860083120313C501C601C701C801C90166
:10018000CA01C40183160313D030810505308104F0
:100190008312031381010030D1000330D3000030FB
:1001A000D4000030D2000030CE0025238316031384
:1001B000061586167730990018111812831203134A
:1001C0009817181318168316031318139816051486
:1001D000831203134B08CC009030D8000130D900B3
:1001E0008C110030CB000030CC00831603130608BE
:1001F0001238860036308312031394004030831681
:1002000003139300831203131308CD008C1183167C
:1002100003138C158B170B17A03083120313DD000B
:100220000030DE0083135E188317831203135D080A
:10023000840055308000DD0A0319DE0A831383121F
:1002400003135E188317831203135D088400FF30C5
:100250008000DD0A0319DE0A8313831203135E187C
:100260008317831203135D08840000308000DD0AC9
:100270000319DE0A8313831203135E188317831294
:1002800003135D088400F7308000DD0A0319DE0ADD
:100290008313831203135E188317831203135D08FD
:1002A000840008308000DD0A0319DE0AA0308312C2
:1002B0000313DD000030DE00AB30E1000030E2006F
:1002C0000030DF0018178C12831603138C168B175F
:1002D0000B172130831203139000E130AC00BD30C6
:1002E000AA00B330AB00AB0B7329AA0B7129AC0B7E
:1002F0006F29000000000000000000000000000066
:1003000000000000000000000000831203130B1126
:10031000831603138B168B170B17831203131010FE
:100320008514A130AC000530AA005E30AB00AB0BE9
:100330009729AA0B9529AC0B932900000000000017
:10034000831203138510CF30AC001F30AA00ED30AC
:10035000AB00AB0BA929AA0BA729AC0BA529000060
:100360000000000000000000000083120313430897
:10037000A1000130A200702083120313A3002318F0
:10038000C229232B831203130C108E018F0110142A
:10039000861583120313051CD729831203130C1C23
:1003A000D6298312031310101F2BD629C9298312B3
:1003B0000313101085146408EC006C08A1000F30C2
:1003C000A2001B20831203132108EC006C08A1007B
:1003D0000730A200752083120313A3002318072AF5
:1003E000831203136C08A1000730A2001B208312A4
:1003F00003132108EC000030D1000330D30000309B
:10040000D4000030D2000230CE002523072A831208
:1004100003136C08A1000030A200702083120313A4
:10042000A3002318142A472A831203136408EB003D
:100430006B08A1001030A2001E20831203132308B2
:10044000EB00EB0A6B08A1000830A20075208312B4
:100450000313A30023183A2A003083120313D10098
:100460000330D3000030D4000030D2000130CE0081
:100470002523472A003083120313D1000430D30010
:100480000030D4000030D2006B08CE002523831248
:1004900003130E08E7000F08E8006708A4006808C7
:1004A000A5002230A6000030A700392083120313D4
:1004B0002808E7002908E8006808E9006708E6005E
:1004C0000030D1000930D3006C08D4000030D200D5
:1004D0000030CE002523003083120313EA000130E0
:1004E000D1000930D3006C08D4000130D200450897
:1004F000CE002523831203136A08A1004508A20039
:100500001120831203132108EA000130D1000930C1
:10051000D3006C08D4000230D2004608CE00252358
:10052000831203136A08A1004608A2001120831257
:1005300003132108EA000130D1000930D3006C0810
:10054000D4000330D2004708CE00252383120313C2
:100550006A08A1004708A200112083120313210892
:10056000EA000130D1000930D3006C08D400043017
:10057000D2004808CE002523831203136A08A10085
:100580004808A2001120831203132108EA00013059
:10059000D1000930D3006C08D4000530D2006908BE
:1005A000CE002523831203136A08A1006908A20064
:1005B0001120831203132108EA000130D100093011
:1005C000D3006C08D4000630D2006608CE00252384
:1005D000831203136A08A1006608A2001120831287
:1005E00003132108EA000130D1000930D3006C0860
:1005F000D4000730D2006A08CE00252300308312D1
:100600000313D1000930D3006C08D4000030D200AD
:100610000130CE002523831203139230AC00113039
:10062000AA003D30AB00AB0B132BAA0B112BAC0B6C
:100630000F2B0000000000008312031385108312AB
:1006400003138611C301B529242B83120313510808
:10065000A1000030A200702083120313A30023180E
:10066000422B83120313CF0A0319D00A8313831278
:10067000031350188317831203134F0884004E0886
:100680008000892B831203135308A1000930A200B4
:10069000702083120313A30023184F2B6C2B83129B
:1006A00003135408A1000830A2000520831203138D
:1006B0002308D4005408A1005208A200112083127C
:1006C00003132108D4005308A1005408A2001120EC
:1006D000831203132108D300903083120313CF0039
:1006E0000130D0004F08A4005008A5005308A60010
:1006F000A7011420831203132408CF002508D0007B
:10070000831350188317831203134F0884004E0875
:10071000800008008C11003083120313CB000030DE
:10072000CC00831603130608123886003630831275
:1007300003139400403083160313930083120313B2
:100740001308CD00080083120313DB01DC018316BC
:100750000313141CC42B83120313DB0A0319DC0AD2
:10076000831203135B08B6005C08B7000030B800C2
:100770000030B900962083120313B5003518C12B41
:10078000C32B8A23F52BA72B83138312031356182D
:10079000831783120313550884000008D700DB0178
:1007A000DC0183120313941357089300941FF22B58
:1007B00083120313DB0A0319DC0A831203135B0899
:1007C000B6005C08B7000030B8000030B9009620D1
:1007D00083120313B5003518EF2BD12BF12B8A238D
:1007E000F52BF22B8312031314160800A03083128A
:1007F0000313DD000030DE00AB30E1000030E2002A
:100800000030DF001A08E0001A08E3000800FF00CB
:10081000030E83120313C0007F08C1002008B2003A
:100820000408831603138C1D1D2C831203138C1DC7
:100830001D2C3C25831203138C11831603138C1E6D
:10084000292C831203138C1E292CF92583120313E0
:100850008C12831603138B1E352C831203130B1D6E
:10086000352C4224831203130B1183120313420805
:1008700084003208A0004108FF00400E8300FF0EF4
:100880007F0E090083120313CA0A4A08B3000E3010
:10089000B4008C2083120313B5003518532C831237
:1008A0000313CA013B2D83120313C90A4908B3007D
:1008B0000230B4008C2083120313B50035183B2D91
:1008C00083120313C9014B08B3004C08B4009120F4
:1008D00083120313B5003518F62C83120313440852
:1008E000B3000530B4008C2083120313B500351813
:1008F000F52C831203130614831603138C118C1228
:10090000831203139401CF30BE001F30BC00ED30C2
:10091000BD00BD0B892CBC0B872CBE0B852C0000A9
:10092000000000000000000000008316031306080A
:1009300036398600831203130608B3003630B4003C
:100940007A2083120313330886002330BE0053300D
:10095000BC00BC0BA92CBE0BA72C831203130608EA
:10096000B300C930B4007D2083120313330886001E
:100970002330BE005330BC00BC0BBC2CBE0BBA2CC9
:100980008C11003083120313CB000030CC0083168F
:1009900003130608123886003630831203139400BE
:1009A0004030831603139300831203131308CD0002
:1009B000831603130615861677309900181118123E
:1009C000831203139817181318168316031318139A
:1009D000981683120313C401831603138C158C1607
:1009E0008312031306100A2DF52CF92C831203131E
:1009F000C40183120313C80A4808B3006330B4006B
:100A00008C2083120313B50035183A2D831203137B
:100A1000C801C40A83120313C70A4708B3003B3056
:100A2000B4008C2083120313B5003518392D8312BE
:100A30000313C701C60A4608B3003B30B4008C203C
:100A400083120313B5003518382D83120313C60122
:100A5000C50A4508B3003B30B4008C208312031351
:100A6000B5003518372D83120313C501372D382DE6
:100A7000392D3A2D3B2D08008316031314088312D9
:100A80000313DA005A08B3002D30B4007D2083121E
:100A900003133308DA005A08B3000930B400912078
:100AA00083120313B5003518E62D831203135A0879
:100AB000B3002930B400912083120313B500351818
:100AC000C52D831203135A08B3000C30B4009120D3
:100AD00083120313B5003518AA2D831203135A0885
:100AE000B3002C30B400912083120313B5003518E5
:100AF0008C2D831203135A08B3002830B4009120C0
:100B000083120313B5003518872D8A238B2D0030EF
:100B100083120313CB00A92D83120313D50A0319E3
:100B2000D60A831203135508B6005608B700EF30F3
:100B3000B8000130B9009F2083120313B5003518A7
:100B4000A82D903083120313D5000130D600A82DB4
:100B5000A323C42D023083120313CB005508B60023
:100B60005608B700831359188317831203135808C4
:100B700084000008B800B9018020831203133608EE
:100B8000D5003708D600A323E52D8312031355089B
:100B9000B6005608B700831359188317831203133E
:100BA000580884000008B800B9018020831203139C
:100BB0003608D5003708D6008313561883178312DA
:100BC00003135508840013088000F82D01308312A8
:100BD0000313CB009030D5000130D6008313591891
:100BE0008317831203135808840080011308CD0073
:100BF000080083120313981CFF2D18121816831275
:100C000003131A08E5008313621883178312031372
:100C100061088400650880006108B6006208B700BA
:100C2000AE30B8000030B900962083120313B5002F
:100C300035181B2E1F2E831203136508DF00831245
:100C400003136108B6006208B700AF30B800003087
:100C5000B9009F2083120313B5003518302E452E9E
:100C6000831203136508B30083135E18831783127E
:100C700003135D0884000008B4009120831203135D
:100C8000B5003518452EF623452E8312031361084F
:100C9000B6006208B700B030B8000030B900962046
:100CA00083120313B5003518562E6A2E83120313D0
:100CB0006508E0006508B400872083120313340838
:100CC000E3005F08B3006508B400892083120313B2
:100CD0003308DF00831203136108B6006208B7000F
:100CE000B130B8000030B900962083120313B5006C
:100CF00035187B2E892E831203136508B300630811
:100D0000B400912083120313B5003518892EF62301
:100D1000892E831203136108B6006208B700B2304F
:100D2000B8000030B900962083120313B5003518BF
:100D30009A2EB12E831203136508B3005F08B40026
:100D4000912083120313B5003518A82EF623A82E80
:100D5000831203136508B400872083120313340839
:100D6000E300831203136108B6006208B700B330D2
:100D7000B8000030B900962083120313B50035186F
:100D8000CC2E83120313DD0A0319DE0A8312031328
:100D9000E10A0319E20AED2E831203136508B3007A
:100DA0006308B400912083120313B5003518D92EBF
:100DB000EC2E831203134308B3000130B4009120DA
:100DC00083120313B5003518EC2E01308312031380
:0C0DD000C3006008E400EC2EF6230800CD
:02400E00022F7F
:00000001FF
